:03000000023104C6
:0C31040078FFE4F6D8FD75814C02314BD9
:100EEC000A53746172743A20004950436F6E6E65F8
:100EFC0063745245510A004950436F6E6E656374BA
:100F0C00003E432C562C43432CC0E4E0EFF2E5F0BA
:100F1C0020D1E8EDEAEEEC49500A003E432C4D415D
:100F2C00432C25303262583A25303262583A2530FB
:100F3C003262583A25303262583A25303262583A89
:100F4C0025303262582C4D414320E0E4F0E5F10AA3
:100F5C00003E432C5645522C20332E3120EEF220ED
:100F6C0025732025732CC2E5F0F1E8FF20495020B1
:100F7C00ECEEE4F3EBFF0A004D61722032382032C4
:100F8C003030380031343A35393A3439003E432C5C
:100F9C004C442C50524F473A202020202020202017
:100FAC002020202020202020202020202020202035
:100FBC002020202020202020202020202020202025
:100FCC002020202020202020202020202020202015
:100FDC00202020202020202020202020202CC4E095
:100FEC00F2E020EFF0EEF8E8E2EAE828F4E0E9EBD2
:100FFC00290A003E2A2C312CCEF1EDEEE2EDFBE578
:10100C0020EFE0F0E0ECE5F2F0FB20F1E5F2E5E2B8
:10101C00EEE3EE20E8EDF2E5F0F4E5E9F1E00A00AC
:10102C003E412C4130312C2562752E2562752E25C2
:10103C0062752E2562752C495020E0E4F0E5F12014
:10104C00E0E4E0EFF2E5F0E00A003E412C41303202
:10105C002C2562752E2562752E2562752E256275DE
:10106C002C495020E0E4F0E5F120EEF1ED2E20F1DA
:10107C00E5F0E2E5F0E00A003E412C4130332C254E
:10108C0062752E2562752E2562752E2562752C498A
:10109C005020E0E4F0E5F120F0E5E72E20F1E5F05A
:1010AC00E2E5F0E00A003E412C4130342C2562751B
:1010BC002E2562752E2562752E2562752CCCE0F1DD
:1010CC00EAE020F1E5F2E80A003E412C4130352CF3
:1010DC002562752E2562752E2562752E2562752C5E
:1010EC00D8EBFEE70A003E532C4130362C256275B6
:1010FC002CC2F0E5ECFF20EEE6E8E42E20EAE2E874
:10110C00F2E0EDF6E8E820282A3130ECF1290A006B
:10111C003E2A2C312CC4EEEF2E20EFE0F0E0ECE573
:10112C00F2F0FB20F1E5F2E5E2EEE3EE20E8EDF281
:10113C00E5F0F4E5E9F1E00A003E422C5330312CA5
:10114C002562752CC6E4E0F2FC20E7E0EFF0EEF14E
:10115C00E020F1EEE5E4E8EDE5EDE8FF20EEF2202D
:10116C00F1E5F0E2E5F0E00A003E422C5330322C7F
:10117C002562752CCEE1ECE5ED20F120F1E5F0E2F5
:10118C00E5F0EEEC20E1E5E720EAE2E8F2E0EDF64E
:10119C00E8E90A003E422C5330332C2562752CCFE3
:1011AC00E5F0E5E7E0EFF3F1EA20EFF0E820EFEE11
:1011BC00F2E5F0E520F1E2FFE7E820F120F1E5F0BF
:1011CC00E2E5F0EEEC0A003E422C5330342C256262
:1011DC00752CCDE5F220EFE5F0E5E4E0F7E820E44E
:1011EC00E8E0E3EDEEF1F2E8EAE820E220F1E5F0E8
:1011FC00E2E5F00A003E422C5330352C2562752C6A
:10120C00CAE0EDE0EB20F8E8F0EEEAEEE2E5F8E01B
:10121C00F2E5EBFCEDEEE3EE20EEE1ECE5EDE00AC1
:10122C00003E532C5330362C253032625825303248
:10123C00625825303262582530326258253032627D
:10124C005825303262582C4D414320E0E4F0E5F152
:10125C0020F8E8F0EEEAEEE2E5F8E0F2E5EBFCED82
:10126C00EEE3EE20EEE1ECE5EDE00A003E454E4407
:10127C000A0044756D70582020202020303020301A
:10128C00312030322030332030342030352030368D
:10129C002030372030382030392030412030422067
:1012AC0030432030442030452030460A003A003A82
:1012BC0020000A0044756D7044202020202030301E
:1012CC002030312030322030332030342030352063
:1012DC003036203037203038203039203041203023
:1012EC00422030432030442030452030460A00450F
:1012FC007272206B657900526420656570726F6D37
:10130C000A005264204D454D0A00526420436F641C
:10131C00650A0044656275674950204F4E0A0044C7
:10132C00656275674950204F46460A0044656275F0
:10133C006755736572204F6E0A0044656275675578
:10134C00736572204F46460A0044656275674D739B
:10135C0067204F6E0A0044656275674D7367204FB6
:10136C0046460A00436F6E666967206C6F636B219B
:10137C000A00577220656570726F6D0A0020536108
:10138C00766520656570726F6D210A00457272205A
:10139C004D414321004C6F61643E3E002A003C41AC
:1013AC0030313D003C4130323D003C4130333D005A
:1013BC003C4130343D003C4130353D003C41303601
:1013CC003D003C21003C5330313D003C5330323D1C
:1013DC00003C5330333D003C5330343D003C5330E3
:0913EC00353D003C5330363D0054
:0638C3000149000147006D
:10392E00C2AFC28E438910758BFF758DB7D2ABD2E5
:04393E008ED2AF2254
:03001B0002306848
:10306800C0E0C083C082C0D0C2AFC28E758BFF756E
:103078008DB720060675A61E75A6E10547D202E59E
:103088004960020549E548D3940140021548054CBA
:10309800E54C540F7050D20EE54C543F701AD200D4
:1030A80090668DE0601204F0E0D394B4400A9080FA
:1030B800007480F0C2AF80FE906688E0600204F081
:1030C800906104E0600214F090668EE0D3940140B1
:1030D80003E014F0300502054AE54BD3946440043C
:1030E800D2068002054BE546D3940140021546D22C
:0C30F8008ED2AFD0D0D082D083D0E03296
:1008A400C291C290D2B5C20B7D027C007F07123880
:1008B400A68F25E525646060097D017F6012385E9E
:1008C400D20BE4FDFC7F0B1238A68F25E52530E61C
:1008D400097D04E4FF123882D20B7D017C007F077E
:1008E4001238A68F25E5257008FD7FFF12385ED2E9
:1008F4000B300B03126000C2AFC288C2A8C2AA7533
:10090400890012341A906341E0B4FA09A3E064CE7A
:1009140070030209A4E4F52574392525F582E4342D
:1009240063F583E4F00525E525B443EC9063417455
:10093400FAF0A374CEF0A374CCF0906347740AF079
:10094400E4A3F0A304F0A3F090634C7403F0A37445
:10095400CCF090633D74FFF0A3F0A3F0E4A3F09017
:1009640063587405F0E4F525E5252401FFE433FE1E
:1009740074392525F582E43463F583E0FD123915D5
:100984000525E525C3944340DFE4F5A775A61E7548
:10099400A6E1907FF0F0A3F09080007480F080FED8
:1009A400D2AF90634C7403F0A374CCF0E490634B27
:1009B400F0122A40C2B5123498C20612372A906344
:1009C40058E0C3940350037403F0D20BC20DC20C5D
:1009D400D293200B077E0E7FEC122561E49065789C
:1009E400F012392EC2AFA37408F09062B77424F0E9
:1009F400E4A3F0906341E09062B9F0906342E09028
:100A040062BAF0906343E09062BBF0906344E0907C
:100A140062BCF0906345E09062BDF0906346E09064
:100A240062BEF0754801E490657AF0C207C208C25C
:100A340009C20AD2AF75A70775A61E75A6E1200BD9
:100A440018AF25FE7D03122762E4FF122F1E7E637A
:100A54007F78E4FB7D0112285C90668DE06003746E
:100A640001F0E4906104F0A37455F0A37481F0E400
:100A7400F54AE4F54B906104E07003122662906637
:100A84008EE0B401119080007410F0E490668EF052
:100A9400D20BC20CC20D908008E0F52530E405D2DB
:100AA400077410F0E52530E508D209908008742019
:100AB400F0E52530E608D2089080087440F0E54A55
:100AC400D394034023908002E4F0908001F090805E
:100AD40000F0E54AD39406400FE4F54AC20390655A
:100AE4007AF075480112372A9080A0E0700312351D
:100AF400139080B8E0700312358D9080D0E07003BD
:100B0400123607908000E0701330071012245D90B5
:100B14006334EFF0D394004003120026908002E087
:100B24007006908000E06005D205020A76C205E4F2
:100B3400F54A906104E06003020A76300912122239
:100B4400F7906334EFF0D394004005E0FF12001FE8
:100B5400200803020CD5122182906334EFF0700355
:100B6400020A76906378E054BF247F7003020C3845
:100B7400147003020C1024026003020C6B200B0798
:100B84007E0E7FF5122561300F7920037690635035
:100B9400E07006906354E0605B906684E0FF9063CD
:100BA40050E0B50724906685E0FE906351E0B506F9
:100BB40018906686E0FE906352E0B5060C90668756
:100BC400E0FE906353E06E602B906354E06F7033EB
:100BD400906685E0FF906355E0B50727906686E050
:100BE400FF906356E0B5071B906687E0FF9063575C
:100BF400E0B5070F90657A7401F012002075480182
:100C0400020CD590668474FFF0020CD590668DE0DA
:100C140060037401F090667CE0FF90637AE06F609B
:100C240003020CD590667CE004F0E4F54890657806
:100C3400F0020CD5300303020CD5906347E0700337
:100C4400020A76123967D203E4F548906578F09089
:100C5400668804F0E490667BF0A3F0200B737E0FAB
:100C64007F03122561806A90668DE060037401F051
:100C7400300352906378E020E74B90637AE0FF9072
:100C8400667BE0FE6F600D906683E07007EE146F84
:100C9400703F801390667BE004F0906334E0FFD3F0
:100CA400940440031232999060007482F0A374019A
:100CB400F090637AE0906002F07E607F007D031222
:100CC400339A020A76300F0920030690668474FF73
:100CD400F0200303020DB1E548706B12395DEF603B
:100CE400207E647F78906479E02404FD12339A9026
:100CF4006683E06003020A76906358E0F548020ACE
:100D040076906688E0D3943C403C906683E07036ED
:100D140090668804F09062B6E0702B122E69E4901D
:100D24006478F0A37412F090667CE090647AF0A387
:100D340074FDF090610763A20190647C63A2017F5B
:100D440012121D54809B1239428F25E525B40115DA
:100D54009060007483F0E4A3F07E607F007D021253
:100D6400339A020A76E525D39401401C90600074FE
:100D740083F0A37401F0E52524FEA3F07E607F00D8
:100D84007D0312339A020A76E54864016003020A7D
:100D940076906578E004F0E0C394055003020CE516
:100DA400C203E490657AF0120020020A76E54864F2
:100DB400016003020A7690657AE014604624FE60BE
:100DC40042147003020E9F24046003020A76E4F5C1
:100DD4004A200F1390657A7404F0906578E054010A
:100DE400F0754801020A769080027410F0E4906570
:100DF4007AF090657804F07548C890668474FFF0C2
:100E0400020A76906684E07003020E8E9064787411
:100E140080F090647A7401F0E4A3F0A304F0A37466
:100E240030F0A3747BF0E4F525747F2525F582E486
:100E34003464F583747DF074802525F582E434648C
:100E4400F583E4F0E5252407906479F07C667D84DD
:100E540090634CE0FAA3E0FB7F021232157E647FBC
:100E640078E5252409FD12339A906683E0601B120D
:100E74003967D203E4F548906578F090668804F009
:100E8400E490667BF0A3F0020A7690657A7404F02D
:100E9400906358E02432F548020A76908002741078
:100EA400F0754803906578E06401FFF090657A740A
:100EB40001F0EF7019906354E06013FCA3E0FDA30C
:100EC400E0FEA3E0FF9066841218E2020A769063C3
:100ED40050E0FCA3E0FDA3E0FEA3E0FF90668412D3
:070EE40018E2020A7680FE0D
:010EEB0022E4
:10002600906379E0B444047F0180027F0090637896
:10003600E0B447047E0180027E00EE5F604A906372
:1000460041E090637AF0906342E090637BF09063C6
:1000560043E090637CF0906344E090637DF09063AE
:1000660045E090637EF0906346E090637FF0906396
:10007600797452F09062B063A2019080A863A201E5
:100086007F06121D5402089A906334E0C394085008
:10009600030208A3906341E0FF90637AE06F600378
:1000A6000208A3906342E0FF90637BE06F60030267
:1000B60008A3906343E0FF90637CE06F600302084F
:1000C600A3906344E0FF90637DE06F60030208A3A2
:1000D600906345E0FF90637EE06F60030208A390A3
:1000E6006346E0FF90637FE06F60030208A39063BE
:1000F60079E0B444159062B0E0B4FF0E63A20190BB
:1001060080A863A2017F06121D5490668DE06003ED
:100116007401F090668E7464F09063797452F09076
:100126006378E0646D60030202A37BFF7A0F790DAA
:100136001214577BFF7A0F7927906341E0F52EA3BF
:10014600E0F52FA3E0F530A3E0F531A3E0F532A307
:10015600E0F533121457752EFF752F0F7530847521
:1001660031FF75320F7533907BFF7A0F795D12146C
:10017600577BFF7A0F79991214577BFF7A0F79FF15
:100186001214577BFF7A10792C906347E0F52EA363
:10019600E0F52FA3E0F530A3E0F5311214577BFF0D
:1001A6007A107956906350E0F52EA3E0F52FA3E080
:1001B600F530A3E0F5311214577BFF7A107984905D
:1001C6006354E0F52EA3E0F52FA3E0F530A3E0F5A8
:1001D600311214577BFF7A1079B290633DE0F52E09
:1001E600A3E0F52FA3E0F530A3E0F5311214577B19
:1001F600FF7A1079D5906339E0F52EA3E0F52FA3A9
:10020600E0F530A3E0F5311214577BFF7A1079F24E
:10021600906358E0F52E1214577BFF7A11791C1261
:1002260014577BFF7A117945A20FE433F52E121489
:10023600577BFF7A117975906683E0F52E12145775
:100246007BFF7A1179A090668DE0F52E1214577B0C
:10025600FF7A1179D39062B6E0F52E1214577BFF20
:100266007A127901A201E433F52E1214577BFF7A34
:1002760012792D90667DE0F52EA3E0F52FA3E0F52B
:1002860030A3E0F531A3E0F532A3E0F533121457BD
:10029600122B267BFF7A12797812145722906378F4
:1002A600E0644C70757E127F7E122561906380E05B
:1002B600F526A3E0F527E4F5297E127FB91225611C
:1002C6007D03AF27AE261227627E127FBB12256101
:1002D600E4F528852782852683E0FF74822528F5A4
:1002E60082E43463F583EFF00527E52770020526DF
:1002F6000528E528B410DC7E637F82E4FB7D1012BE
:10030600285C7E127FBE1225610529E529C394105B
:1003160040A77E127FBE12256122906378E0646C4E
:10032600705CF52A7E127FC0122561E4F529AF2A9A
:100336007E007D031227627E127FBB122561E4F5E3
:1003460028A82AE6FF74822528F582E43463F5831B
:10035600EFF0052A0528E528B410E67E637F82E4DF
:10036600FB7D1012285C7E127FBE1225610529E5F1
:1003760029C3940840B87E127FBE1225612290637D
:1003860078E0644B7061F528746A2528F582E434B8
:1003960063F583E06032746A2528F582E43463F5F8
:1003A60083E0F46023746A2528F582E43463F583D8
:1003B600E0FF74802528F582E43463F583E0B50711
:1003C600100528E528B408C09061047432F00208CC
:1003D6009A9063787421F0300B0302089A7E127F9C
:1003E600FB12256102089A906378E0B4521A200B3A
:1003F600077E137F031225619063787472F07E6323
:100406007F787D0812331A22906378E0644970453C
:10041600200B077E137F0E122561906380E0F52680
:10042600A3E0F527E4F528852782852683E0FF7477
:10043600822528F582E43463F583EFF00527E52766
:10044600700205260528E528B480DC7E637F787D6A
:100456008A12331A22906378E064437079A3E064C9
:10046600527046200B077E137F161225619063801B
:10047600E0F526A3E0F527E4F5288527828526837F
:10048600E493FF74822528F582E43463F583EFF064
:100496000527E527700205260528E528B480DB7EBA
:1004A600637F787D8A12331A22906379E0645760FD
:1004B600030208A3906380E0F526A3E0F527748283
:1004C6002528F582E43463AD82FC7B80AF27AE2617
:1004D60012380202089A906378E0644460030205C9
:1004E6006D906380E0FF6444700302089AEFB431B4
:1004F6000CC20B7E137F1F12256102089A9063803F
:10050600E0B4300CD20B7E137F2B12256102089AC1
:10051600906380E0B4320CD20C7E137F38122561D2
:1005260002089A906380E0B4330CC20C7E137F46B7
:1005360012256102089A906380E0B4340CD20D7ED5
:10054600137F5512256102089A906380E0B4350C3A
:10055600C20D7E137F6212256102089A906380E0C5
:10056600FF12001E02089A906104E07013200B0728
:100576007E137F701225619063787421F002089AC9
:100586009061047432F0906378E0FFB4510A908071
:10059600007480F0C2AF80FEEF64577045200B07F1
:1005A6007E137F7E122561906381E0906334F0E4D0
:1005B600F528906334E0FFE528C39F400302089ABC
:1005C60074822528F582E43463F583E0FF90638026
:1005D600E0252824AFF582E43461F583EFF00528A1
:1005E60080D0906378E06453600302069C200B077A
:1005F6007E137F89122561906341E0FF9061B8E028
:100606006F703C906342E0FF9061B9E06F7030908C
:100616006343E0FF9061BAE0B50724906344E0FFCE
:100626009061BBE0B50718906345E0FF9061BCE0C0
:10063600B5070C906346E0FF9061BDE06F601690D1
:1006460063787421F0300B0302089A7E137F9812A8
:10065600256102089AE4F528E4F54BAF28FE74AF4D
:100666002528F582E43461F583E0FD123915052865
:10067600E528C394FE40E19080007480F0C2AFE4A8
:10068600907FF0F0A3F0907FFD74AAF0A374FFF0C2
:10069600A37455F080FE906378E0644F704C9063CD
:1006A60080E0F526A3E0F527E5274526700A200B0E
:1006B600077E137FA1122561200B077E137FA812E8
:1006C6002561E4F52874822528F582E43463F583F0
:1006D600E0852782852683F00527E5277002052613
:1006E6000528E528B480DE02089A906378E0FFB416
:1006F60045279080007480F0906380E0FDA3E09031
:100706007FF0CDF0A3EDF0C2AF907FFD74AAF0A309
:1007160074FFF0A37455F080FEEF64656003020871
:100726009A906380E0FFA3E0907FF0CFF0A3EFF014
:10073600E4F526F527D3907FF1E09527907FF0E04A
:1007460095264020E4F54B2527FFE5263401FE8556
:100756002782852683E0FD1239150527E5277002D5
:10076600052680D17E137FAA123190EF4E602012AB
:100776000003906347EFF0120003906348EFF01216
:100786000003906349EFF012000390634AEFF07E96
:10079600137FB0123190EF4E602012000390635029
:1007A600EFF0120003906351EFF0120003906352D2
:1007B600EFF0120003906353EFF07E137FB6123111
:1007C60090EF4E6020120003906354EFF012000386
:1007D600906355EFF0120003906356EFF01200039A
:1007E600906357EFF07E137FBC123190EF4E60207E
:1007F60012000390633DEFF012000390633EEFF0AA
:1008060012000390633FEFF0120003906340EFF095
:100816007E137FC2123190EF4E6020120003906368
:1008260039EFF012000390633AEFF0120003906381
:100836003BEFF012000390633CEFF07E137FC8128B
:100846003190EF4E60081236CD906358EFF0E4F524
:1008560028E4F54BE5282401FFE433FE7439252806
:10086600F582E43463F583E0FD1239150528E528A1
:10087600C3944340DC9080007480F0C2AFE4907F64
:10088600F0F0A3F0907FFD74AAF0A374FFF0A374B8
:0D08960055F080FE7E637F787D0812331AD6
:0108A3002232
:1037CA00AE07EEC39430400BEED394395005EE2485
:1037DA00D0FF22EEC39461400BEED394665005EEFF
:1037EA0024A9FF22EEC39441400BEED39446500520
:0837FA00EE24C9FF22AF0622F4
:1038FB009062AFE004F070069062AEE004F090626C
:0A390B00AEE0FEA3E0FF1238DF2259
:100003001238FB1237CAEFC454F0FEC0061238FB95
:080013001237CAD0E02FFF22D2
:1036CD00E49069B7F01238FB9069B8EFF0C394300D
:1036DD004018E0FFD3943950119069B7E02407F5F5
:1036ED0082E43461F583EFF080119069B7E024072F
:1036FD00F582E43461F583E4F0800C9069B7E00461
:10370D00F0E0D3940840BE752E00752F0075300083
:0C371D00E4F5317B017A617907121E622D
:01372900227D
:043190008E2B8F2CC7
:103194009062AEE4F0A374FFF01238FBEF606EF4BB
:1031A400606B852C82852B83E493B507EC752D0128
:1031B400E52C252DF582E4352BF583E493602590E9
:1031C40062AFE0252DFF9062AEE03400FE1238DFDE
:1031D400E52C252DF582E4352BF583E493B507041E
:1031E400052D80CCE52C252DF582E4352BF583E4E3
:1031F4009370A6E52D24FFFFE434FFFE9062AFE058
:103204002FF09062AEE03EF07E007F0122E4FEFFEC
:013214002297
:102A40007E137FCE123190EF4E70037F01227E13F2
:102A50007FD1123190EF4E600C1238FBEF24D0245E
:102A6000FF920F8002D20F7E137FD7123190EF4E6C
:102A7000600C1238FBEF24D0906683F08005E49060
:102A80006683F07E137FDD123190EF4E600C1238BA
:102A9000FBEF24D090668DF08005E490668DF07E8B
:102AA000137FE3123190EF4E600C1238FBEF24D00D
:102AB0009062B6F08005E49062B6F07E137FE91272
:102AC0003190EF4E600C1238FBEF24D024FF9201BE
:102AD0008002C20190634163A20190667D63A201FE
:102AE0007F06121D5430013B7E137FEF123190EFB1
:102AF0004E603012000390667DEFF0120003906686
:102B00007EEFF012000390667FEFF01200039066F4
:102B100080EFF0120003906681EFF01200039066E0
:062B200082EFF07F0022AD
:10378300906579E0C3947C503D906579E0FE04F048
:1037930074B72EF582E43462F583EFF0BF0A279005
:1037A3006579E0FF04F074B72FF582E43462F583A2
:1037B300E4F0906579E0FF122FC89065797408F002
:0737C3009062B8E004F0225F
:10372A009080007480F090633963A201F583F5827A
:10373A0063A2017F08121D5490634163A201908025
:10374A008863A2017F0A121D54908092E4F0A37448
:10375A0032F0A37401F090634BE0FF9080B1F090D7
:10376A0080E1EFF09080957455F0A3F0908000749A
:09377A0001F090800974F0F022C6
:10351300908009E04410F09080A0E0706C9080A14E
:103523007482F09080A874FFF0A3F0A3F0A3F07F5F
:10353300039080AEEFF07FCBA3EFF07F039080ACDE
:10354300EFF0A374CBF09080007402F09069A7129F
:1035530018EE000000009069A7E0908040F09069A9
:10356300A8E0908041F09069A9E0908042F09069D2
:10357300AAE0908043F0A3E4F0A3F0A3F0A3F090BB
:093583008018F0A3F0A3F0A3F0FE
:01358C00221C
:10360700908009E04440F09080D17482F090634C40
:10361700E0FF9080DEF090634DE0FF9080DFF09058
:1036270080027402F09069AB1218EE00000000905F
:1036370069ABE0908058F09069ACE0908059F090C9
:1036470069ADE090805AF09069AEE090805BF0A39E
:10365700E4F0A3F0A3F0A3F0908030F0A3F0A3F080
:02366700A3F0CE
:01366900223E
:10358D00908009E04420F09080B8E0706C9080B994
:10359D007482F07F039080C6EFF07FCDA3EFF07FB4
:1035AD00039080C4EFF0A374CDF09080C074FFF051
:1035BD00A3F0A3F0A3F09080017402F09069AF1214
:1035CD0018EE000000009069AFE090804CF090691B
:1035DD00B0E090804DF09069B1E090804EF0906930
:1035ED00B2E090804FF0A3E4F0A3F0A3F0A3F0902D
:0935FD008024F0A3F0A3F0A3F078
:0136060022A1
:103215008C268D27A907EAFDE975F018A424ACFFD3
:10322500E5F034808F82F583EDF0EBFDE975F0185C
:10323500A4FFAEF024ACFBEE34808B82F583A3EDC6
:10324500F08527828C83E0FDEF24A8FFEE3480FE15
:103255008F82F583EDF08527828C83A3E08F828EA4
:1032650083A3F0852782852683A3A3E0FDE975F076
:1032750018A424A8FFE5F03480FE8F82F583A3A36C
:10328500EDF08527828C83A3A3A3E08F828E83A391
:04329500A3A3F022DD
:06331A008D2BAB07AA0693
:10332000908000E020E5729069A7E0FCA3E0FDA397
:10333000E0FEA3E0F52F8E2E8D2D8C2CAE02AF0378
:103340008E838F8263A201E52E540744C0F58385E6
:103350002F8263A201AF2B121DC6E4FCFDFEE52FF8
:10336000252BF52FEE352EF52EED352DF52DEC35E3
:103370002CF52C908040E52CF0A3E52DF0A3E52E54
:10338000F0A3E52FF09080007420F0AF2FAE2EADAB
:093390002DAC2C9069A71218E283
:013399002211
:06339A008D26AB07AA0618
:1033A000908002E020E5729069ABE0FCA3E0FDA311
:1033B000E0FEA3E0F52A8E298D288C27AE02AF030C
:1033C0008E838F8263A201E529540744D0F583855B
:1033D0002A8263A201AF26121DC6E4FCFDFEE52A87
:1033E0002526F52AEE3529F529ED3528F528EC3581
:1033F00027F527908058E527F0A3E528F0A3E529D5
:10340000F0A3E52AF09080027420F0AF2AAE29AD37
:0934100028AC279069AB1218E208
:013419002290
:022F1E008F26FC
:102F2000908001E030E5037F00229069AFE0FCA3D0
:102F3000E0FDA3E0FEA3E0F52A8E298D288C2790E2
:102F4000667D63A201E529540744C8F583852A827A
:102F500063A2017F06121DDCE52A2406F52AE4356A
:102F600029F529E43528F528E43527F52790657BF0
:102F700063A201E529540744C8F583852A8263A228
:102F800001AF26121DDCE4FCFDFEE52A2526F52A0C
:102F9000EE3529F529ED3528F528EC3527F527906C
:102FA000804CE527F0A3E528F0A3E529F0A3E52A66
:102FB000F09080017420F0AF2AAE29AD28AC2790A4
:072FC00069AF1218E2AF2611
:012FC70022E7
:10245D009081E0E0F52605260526052605260526AC
:10246D0005260526052605260526908010E0F5296A
:10247D00A3E0F52AA3E0F52BA3E0F52C9081E1E094
:10248D00F5260526052605260526052605260526F7
:10249D00052605260526908014E0F52DA3E0F52EE2
:1024AD00A3E0F52FA3E0F530E52FB52B08E530B50A
:1024BD002C037F0022E4F526E52F540744E0F58335
:1024CD0085308263A20190637863A2017F08121E9A
:1024DD000C90637A63A2019062B063A2017F061231
:1024ED001D54906378E0F527A3E0F528E4F52690D8
:1024FD006378E0702AA3E024F8F526E52F5407440D
:10250D00E0F58385308274082582F582E43583F504
:10251D008363A20190637863A201AF26121E0CAEF5
:10252D0027E4FCFDE5302528F530E52F3EF52FEDB0
:10253D00352EF52EEC352DF52D908014E52DF0A3CF
:10254D00E52EF0A3E52FF0A3E530F0908000744068
:03255D00F0AF26B6
:012560002258
:102182009081E6E0F5260526052605260526052684
:1021920005260526052605260526908028E0F52930
:1021A200A3E0F52AA3E0F52BA3E0F52C9081E7E06C
:1021B200F5260526052605260526052605260526D5
:1021C20005260526052690802CE0F52DA3E0F52EA8
:1021D200A3E0F52FA3E0F530E4F526E52FB52B0AB1
:1021E200E530B52C05C2080222DCE52F540744F085
:1021F200F58385308263A20190637863A2017F0830
:10220200121E0C906378E0F527A3E0F528E5284537
:102212002770099080027410F07F0022906684E09B
:10222200FFF4602D90637AE06F7076906685E0FF30
:1022320090637BE06F706A906686E0FF90637CE05B
:102242006F705E906687E0FF90637DE06F60228032
:102252005090637AE0906684F090637BE0906685AC
:10226200F090637CE0906686F090637DE0906687F4
:10227200F0906378E0702AA3E024F8F526E52F5465
:102282000744F0F58385308274082582F582E435AF
:1022920083F58363A20190637863A201AF26121EC5
:1022A2000CAE27E4FCFDE5302528F530E52F3EF5A0
:1022B2002FED352EF52EEC352DF52DAF2CAE2BADA9
:1022C2002AAC29AB30AA2FA92EA82DD31218D1409F
:1022D200099080027410F07F002290802CE52DF08E
:1022E200A3E52EF0A3E52FF0A3E530F09080027471
:0422F20040F0AF26E3
:0122F60022C5
:1022F7009081E3E0F5260526052605260526052611
:102307000526052605260526052690801CE0F529C5
:10231700A3E0F52AA3E0F52BA3E0F52C9081E4E0F8
:10232700F52605260526052605260526052605265E
:10233700052605260526908020E0F52DA3E0F52E3D
:10234700A3E0F52FA3E0F530E4F526E52FB52B0A3A
:10235700E530B52C05C209022442E52F540744E8AD
:10236700F58385308263A20190600463A2017F0E2A
:10237700121E22906004E0F527A3E0F52890600C78
:10238700E0FFF4604590667DE0FEEF6E706EA3E0BF
:10239700FF90600DE06F706490667FE0FF90600EC5
:1023A700E06F7058906680E0FF90600FE06F704CB0
:1023B700906681E0FF906010E06F7040906682E069
:1023C700FF906011E06F60048032D2D9906004E022
:1023D700702AA3E024F2F526E52F540744E8F58395
:1023E700853082740E2582F582E43583F58363A2F6
:1023F7000190600463A201AF26121E22AE27E4FCFF
:10240700FDE5302528F530E52F3EF52FED352EF586
:102417002EEC352DF52DAF2CAE2BAD2AAC29AB30DC
:10242700AA2FA92EA82DD31218D15006E528452783
:1024370070099080017410F07F0022908020E52DB4
:10244700F0A3E52EF0A3E52FF0A3E530F09080018F
:052457007440F0AF2607
:01245C00225D
:042561008E2B8F2C02
:10256500E4F52DF52E908000E030E511052EE52EE1
:102575007002052DD39488E52D941340E8908000D2
:10258500E030E5030226619069A7E0FCA3E0FDA326
:10259500E0FEA3E0F5328E318D308C2FE532FFE57C
:1025A500315407FEE42FF52EEE34C0F52D852E822D
:1025B500F5837423F0052EE52E7002052D532DC7E6
:1025C500F582852D83740AF0052EE52E7002052D02
:1025D500532DC790634163A201852D83852E8263A8
:1025E500A2017F06121DC67406252EF52EE4352D93
:1025F500F52D852B83852C8263A201852D83852E60
:102605008263A201121DAAE4FCFDFE9069A7E0F811
:10261500A3E0F9A3E0FAA3E02FFFEE3AFEED39FDC2
:10262500EC38FCEF2408FFE43EFEE43DFDE43CFC11
:102635009069A71218E29069A7E0908040F0906930
:10264500A8E0908041F09069A9E0908042F09069FF
:0C265500AAE0908043F09080007420F018
:012661002256
:06285C008E2B8F2C8D2D48
:10286200E4F52EF52F908000E030E511052FE52FDD
:102872007002052ED39488E52E941340E8908000D0
:10288200E030E50302294F9069A7E0FCA3E0FDA335
:10289200E0FEA3E0F5338E328D318C30E533FFE577
:1028A200325407FEE42FF52FEE34C0F52E852F8229
:1028B200F5837423F0052FE52F7002052E532EC7E2
:1028C200F582852E83EBF0052FE52F7002052E533E
:1028D2002EC790634163A201852E83852F8263A256
:1028E200017F06121DC67406252FF52FE4352EF53D
:1028F2002E852B83852C8263A201852E83852F82D0
:1029020063A201AF2D121DC67408252DF52DFFE41B
:10291200FCFDFEE5332FF533EE3532F532ED353180
:10292200F531EC3530F530908040E530F0A3E531FB
:10293200F0A3E532F0A3E533F09080007420F0AF0D
:0D29420033AE32AD31AC309069A71218E20F
:01294F002265
:022FC8008F3F39
:102FCA00E4F540F541908000E030E5110541E54126
:102FDA0070020540D39488E540941340E89080003D
:102FEA00E020E5799069A7E0FCA3E0FDA3E0FEA359
:102FFA00E0F5458E448D438C42E545FFE544540790
:10300A00FEE42FF541EE34C0F5409062B763A201A9
:10301A0085408385418263A201AF3F121DC6E4FC4D
:10302A00FDFEE545253FF545EE3544F544ED3543CE
:10303A00F543EC3542F542908040E542F0A3E54382
:10304A00F0A3E544F0A3E545F09080007420F0AFCA
:0D305A0045AE44AD43AC429069A71218E2A8
:013067002246
:062762008E2B8F2CAB054D
:10276800E4F52DF52E908000E030E511052EE52EDC
:102778007002052DD39488E52D941340E8908000CD
:10278800E030E50302285B9069A7E0FCA3E0FDA325
:10279800E0FEA3E0F5328E318D308C2FE532FFE577
:1027A800315407FEE42FF52EEE34C0F52D852E8228
:1027B800F5837423F0052EE52E7002052D532DC7E1
:1027C800F582852D83EBF0052EE52E7002052D9000
:1027D800634163A201852D83852E8263A2017F0652
:1027E800121DC67406252EF52EE4352DF52D532D14
:1027F800C7E52B852E82852D83F0052EE52E7002E8
:10280800052D532DC7F582852D83E52CF0052EE582
:102818002E7002052D532DC7E532240AF532E43512
:1028280031F531E43530F530E4352FF52F9080401F
:10283800E52FF0A3E530F0A3E531F0A3E532F09001
:1028480080007420F0AF32AE31AD30AC2F9069A764
:032858001218E271
:01285B00225A
:10366A00908009E04480F09080E97401F07F09902D
:10367A0080F6EFF0A37464F09080037402F09080F7
:10368A0000E020E1F99068A31218EE000000009013
:10369A0068A3E0908064F09068A4E0908065F09060
:1036AA0068A5E0908066F09068A6E0908067F0A335
:1036BA00E4F0A3F0A3F0A3F090803CF0A3F0A3F011
:0236CA00A3F06B
:0136CC0022DB
:102C0B009081E9E0F52705270527052705270527E7
:102C1B0005270527052705270527908034E0F5288C
:102C2B00A3E0F529A3E0F52AA3E0F52B9081EAE0D8
:102C3B00F527052705270527052705270527052739
:102C4B00052705270527908038E0F52CA3E0F52D07
:102C5B00A3E0F52EA3E0F52FE52EB52A08E52FB559
:102C6B002B037F0022AF2FAE2EAD2DAC2CAB2BAA9E
:102C7B002AA929A828D31218D1400AAF2FAE2BEEC0
:102C8B009FF527800AAF2FEFF404AE2B2EF527E527
:102C9B002E540744E0F583852F8263A2019068A729
:102CAB0063A201AF27121E3AE4FCFDFEE52F252798
:102CBB00F52FEE352EF52EED352DF52DEC352CF5BE
:102CCB002C908038E52CF0A3E52DF0A3E52EF0A396
:0B2CDB00E52FF09080037440F0AF275D
:012CE60022CB
:022950008F27CF
:102952009080E8E0640660037FFF229068A3E0FCB9
:10296200A3E0FDA3E0FEA3E0F52B8E2A8D298C289F
:10297200E4FFFEFDFCAB2BAA2AA929A828C3121842
:10298200D170609081F9E0F5289068A3E0FCA3E0A3
:10299200FDA3E0FEA3E0FFE4FAF9F8EF2401FFEA69
:1029A2003EFEE93DFDE83CFC9068A31218E2906807
:1029B200A3E0FCA3E0FDA3E0FEA3E0FFE4F8EF2424
:1029C20001FFEA3EFEE93DFDE83CFC9068A31218D7
:1029D200E2908064E0F528A3E0F529A3E0F52AA3BC
:1029E200E0F52B9068A763A201E52A540744D8F5C5
:1029F20083852B8263A201AF27121DF4E4FCFDFE46
:102A0200E52B2527F52BEE352AF52AED3529F52973
:102A1200EC3528F528908064E528F0A3E529F0A399
:102A2200E52AF0A3E52BF09080037420F0AF2BAEE3
:0D2A32002AAD29AC289068A31218E27F009D
:012A3F002274
:1038DF00E5D220E0FBC2AF438E2075D2028F828EDD
:0B38EF0083E0FFE4F5D2538EDFD2AF80
:0138FA0022AB
:10391500E5D220E0FBC2AF43D2028F828E83EDF069
:0939250075D25063D250D2AF22DA
:10341A00E4FDED2401FFE433FE1238DF74392DF5A3
:10342A0082E43463F583EFF00DBD3FE6E4FDED245D
:10343A007FFFE433FE1238DF742F2DF582E4346106
:10344A00F583EFF0742F2DF582E43461F583E07093
:10345A001B742F2DF582E43461F5837420F07430E7
:10346A002DF582E43461F583E4F080040DBD80BE5D
:10347A00E49061AEF0FDEDFF7E001238DF74AF2DEF
:0D348A00F582E43461F583EFF00DBDFEE93D
:013497002212
:023802008B2B0E
:10380400A2AF9219C2AF85A22C53A2FE8E838F82DF
:1038140005A28C838D827409121E50E52B53A2FEDF
:1038240043A220121E5253A2DF852CA2A21992AFEA
:01383400FF94
:013835002270
:1038A600A2AF9219C2AF8C838D82EF121E5043A233
:0C38B60020121E5253A2DFA21992AFFF95
:0138C20022E3
:02385E008F26B3
:10386000A2AF9219C2AFE4F5838D827406121E5086
:10387000E52643A220121E5253A2DFA21992AF7F67
:013880000146
:013881002224
:023882008F268F
:10388400A2AF9219C2AFE4F5838D82740A121E505E
:10389400E52643A220121E5253A2DFA21992AF7F43
:0138A4000122
:0138A5002200
:101C7900A907E7FFA805EF93C3966008403B74FCEA
:101C89002FFF80F00F08EF93C3966008402B74FB79
:101C99002FFF80E00F08EF93C3966008401B74FA8A
:101CA9002FFF80D00F08EF93D3966008400B74F98B
:101CB9002FFF80C01F1F1F1F1FEF54FEF80303F7DC
:101CC900E893FC08E893FD08E893FE08E893FF22EF
:101CD90009E993C39D6008402974FB29F980F1093A
:101CE900E993C39E6008401A74FA29F980E209E968
:101CF90093D39F6008400B74F929F980D3191919F6
:101D09001919E9C313C313FF22740093F8ECC3989C
:101D19004024701F740193F8EDC39840197014742E
:0E1D29000293F8EEC398400E7009740393F80D
:101D3700EFC39840037F00227F0122EDF8E6F00809
:101D4700A3DFFA22EDF8E0F608A3DFFA22E0A363A7
:101D5700A201F0A363A201DFF475A2002263A2012E
:101D6700F0A363A20122E0A363A201F0A363A2018F
:101D7700E0A363A201F0A363A201E463A201F0A3BD
:101D870063A201DFE175A20022E0A363A2016DFE59
:101D9700936CFDEE058393FC158363A201DFEA755F
:101DA700A200227F00E493A363A201F00F600CA3BB
:101DB700E583C2E3F58363A20180EA75A20022E00E
:101DC700A363A201F0A3E583C2E3F58363A201DF66
:101DD700EE75A20022E0A363A201F0A3E583C2E4AB
:101DE700D2E3F58363A201DFEC75A20022E0A363CF
:101DF700A201F0A3E58344F8C2E5F58363A201DFFE
:101E0700EC75A20022E583C2E3F583E0A363A20198
:101E1700F0A363A201DFEE75A20022E583C2E4D23C
:0A1E2700E3F583E0A363A201F0A33A
:101E310063A201DFEC75A20022E58344F8F583E09B
:101E4100A363A201F0A363A201DFEE75A20022F950
:101E510022C002C004C00612FFF0D006D004D00296
:011E6100225E
:101A17003E2A2C312CCFE0F0E0ECE5F2F0FB20E0A1
:101A2700F1E8EDF5F0EEEDEDEEE3EE20EFEEF0F29E
:101A3700E00A003E4C2C4930312C256C752CD1EA3C
:101A4700EEF0EEF1F2FC20EEE1ECE5EDE02C3530C6
:101A57002C3130302C3330302C3630302C31323082
:101A6700302C323430302C343830302C393630305A
:101A77002C31393230302C33383430302C3537363E
:101A870030302C3131353230300A003E422C49306B
:101A9700322C2562752CCFF0EEE2E5F0FFF2FC2048
:101AA70043545320EFF0E820EFE5F0E5E4E0F7E5F5
:101AB7000A003E532C4931312C25752CC7E0E4E54B
:101AC700F0E6EAE020F1F2E0F0F2E020EFE5F0E501
:101AD700E4E0F7E82028ECF1290A003E4C2C4930D5
:101AE700342C25732CD0E5E6E8EC20EFE5F0E5E4AF
:101AF700E0F7E82C3820E1E8F22C3720E1E8F20A99
:101B0700003820E1E8F2003720E1E8F2003E4C2CF3
:101B17004931302C25732CCAEEEDF2F0EEEBFC20A8
:101B2700F7E5F2EDEEF1F2E82C302DCDE5F22C31B0
:101B37002DD7E5F2EDFBE920284556454E292C32F5
:101B47002DCDE5F7E5F2EDFBE920284F4444290ABE
:101B570000302DCDE5F200312DD7E5F2EDFBE92080
:101B6700284556454E2900322DCDE5F7E5F2EDFB28
:101B7700E920284F444429003E532C4930372C256F
:101B870062752CC4EEF1F2E0E2EAE020EFF0E82023
:101B9700EFF0E8E5ECE5204E20E1E0E9F220283C13
:101BA700313236290A003E532C4930392C256275CB
:101BB7002CC4EEF1F2E0E2EAE020EFF0E820EFF0EB
:101BC700E8E5ECE520E1E0E9F2E02028302DEDE55D
:101BD700F220EAEEEDF2F0EEEBFF290A003C493085
:101BE700313D003C4930323D003C4930333D003CFB
:101BF7004931313D003C4930343D003C4930353DA9
:101C0700003C4930363D003C4931303D003C4930CD
:101C1700373D003C4930393D000AC1F3F4E5F02077
:101C2700E7E0EDFFF221000A2D3E000A4672616DE2
:101C370065206572726F722120000A3C2D00496E83
:101C470069745443500A004C697374656E54435069
:101C57000A00534F434B5F5443505F45535441422F
:101C67004C49534845440A000A2D3E20000A3C2DA2
:021C770020004B
:1038C90052668F00000000000000000000000000A8
:0538D9000000000000EA
:01001E0022BF
:03002300022DA902
:0B2DA900C0E0C083C082C0D075D0180D
:102DB400309841E50D25E9F5EB30D709E50C25F907
:102DC40004F5FB8006E50C25F9F5FBAF99D2917467
:102DD400A12510F582E43466F583EFF00510E50EC5
:102DE4006005B51F02D2D9E510547FD3950840027F
:102DF400D2D9C298309965301260301707309704E1
:102E0400D2108056E512C3950F400AC212C290D266
:102E140018D2968045AF12051274A12FF582E434BE
:102E240067F583E0F51530151953157F3011282007
:102E3400D008201422631580801D30141A63158075
:102E44008015301112E5155215301406A2D0929B4C
:0C2E54008005A2D0B3929B851599C2990D
:092E6000D0D0D082D083D0E03242
:102B26007BFF7A1A79171214579068A1E0FEA3E08A
:102B3600FFC3E49FFFE49EFEAB07FA3395E0F9F886
:102B46007F007E8C7D0A7C001218318F318E308D8D
:102B56002F8C2E7BFF7A1A793A1214577BFF7A1A3A
:102B66007992A217E433F52E121457AE09AF0A7CF8
:102B7600007D0A1217518E2E8F2F7BFF7A1A79B994
:102B8600121457201514752EFF752F1B7530087BF0
:102B9600FF7A1A79E21214578012752EFF752F1BD1
:102BA60075300E7BFF7A1A79E212145720111475CC
:102BB6002EFF752F1B7530587BFF7A1B7914121464
:102BC600578029301414752EFF752F1B75305E7BC8
:102BD600FF7A1B79141214578012752EFF752F1B5E
:102BE60075306E7BFF7A1B79141214577BFF7A1BA4
:102BF600797F85082E1214577BFF7A1B79AD850ED7
:052C06002E12145722FC
:102006007E1B7FE4123190EF4E600B1236CD906945
:10201600B31218E2800A9069B31218EE0000258008
:102026009069B3E0F8A3E0F9A3E0FAA3E0FB7F0030
:102036007E8C7D0A7C001218311218C39068A1EEBE
:10204600F0A3EFF0E47B0AFAF9F89069B3E0FCA399
:10205600E0FDA3E0FEA3E0FF121831A804A905AA3B
:1020660006AB07E47FB87E88FDFC1218318E0C8F14
:102076000D7E1B7FEA123190EF4E600C1238FBEF9B
:1020860024D024FF92178002C2177E1B7FF01231E4
:1020960090EF4E60121236CDE47B64FAF9F812170F
:1020A600A68E098F0A8005E4F509F50A7E1B7FF6E0
:1020B600123190EF4E60121236CDE47B0AFAF9F82F
:1020C6001217A68E098F0A8005E4F509F50A7E1B0C
:1020D6007FFC123190EF4E600A1238FBEF24D0F5E8
:1020E600158003751508E515B40704D2158002C2DC
:1020F600157E1C7F02123190EF4E600C1238FBEFFA
:1021060024D024FF92118002C2117E1C7F08123156
:1021160090EF4E600C1238FBEF24D024FF9214800F
:1021260002C2147E1C7F0E123190EF4E600A1238E6
:10213600FBEF24D0F5158005E4F515C211E515B4BD
:102146000104D211D214E515B40204D211C2147ED0
:102156001C7F14123190EF4E60071236CD8F088027
:10216600037508407E1C7F1A123190EF4E600712ED
:0B21760036CD8F0E8003E4F50E7F00D5
:01218100223B
:10383600C2A9438902758C48758A4875D90475DB17
:103846004875DC4875DD4875DE48E4F5E9F5F9C2EA
:08385600D9C2DAD28CD2DE22C5
:10349800C212C218E4F512F50FF510C210D297D275
:1034A80096751309122006C2ADE4F5C9D2CDD2CC67
:1034B800C2C9C2CAF5CDF5CC9068A1E0F5CBA3E0AE
:1034C800F5CA85CBCD85CACCE4F59830110C20150A
:1034D800095387BFD29FD29E8002D29E438740C2A3
:1034E8009FC2ACC298C29975B81075B710D2CAD22B
:1034F8009CD2AC123836C2D9E5E92464F5EB30D752
:0B35080006E5F904F5FB2285F9FB2223
:01001F0022BE
:102E6900E4FF0F2407F582E43461F583E513F00FDD
:102E790074072401F582E43461F583E4F07C667D0E
:102E890094FEED1DAA0470011CF5828A83E0FBAA59
:102E9900070F74072AF582E43461F583EBF00EBE5F
:102EA90004E07C667D98E4FEED1DAA0470011CF522
:102EB900828A83E0FBAA070F74072AF582E434614A
:102EC900F583EBF00EBE04E07C667D9CE4FEED1D0F
:102ED900AA0470011CF5828A83E0FBAA070F740714
:102EE9002AF582E43461F583EBF00EBE04E07C66DA
:102EF9007DA0E4FEED1DAA0470011CF5828A83E021
:102F0900FBAA070F74072AF582E43461F583EBF015
:042F19000EBE04E004
:012F1D002291
:0A395300C2992099FDD299D290226A
:07396700D2CAD29CD2AC22AF
:103299008F2620167B30120B200B757E1C7F201287
:1032A90025612290637BE0F513E52624FCFFF50FE9
:1032B9007D7C758363058263A2019067A163A20186
:1032C900121D54E4F512D212C296301702D210E53B
:1032D9000A4509601EC2DAE50A25E9F5EC30D70985
:1032E900E50925F904F5FC8006E50925F9F5FCD27F
:1032F900138003123953200B157E1C7F2E12256172
:103309007E677FA1E52624FCFDE4FB12285CC21838
:013319002291
:102CE70020D9037F0022C2D9E5E92410F5EB30D7BC
:102CF70008E5F92428F5FB8006E5F92427F5FBE527
:102D070010547FD394005003022DA6C291C2AF8501
:102D17001014631080531080D2AF30161DE5145481
:102D27008024A1F582E43466F58363A2019068A745
:102D370063A201AF14121D54805DE4906478F0E53E
:102D470014547FFFA3F090667CE090647AF0A3E5CB
:102D570013F0E514548024A1F582E43466F5836307
:102D6700A20190647C63A201121D54200B29309F9D
:102D7700077E1C7F321225617E1C7F41122561E58B
:102D870014548024A1F582E43466AF82FEE514541E
:102D97007FFDE4FB12285CC29FE514547FFF227F6E
:022DA700002208
:0100200022BD
:102662003000489080E8E0700F12366A300D077E25
:102672001C7F45122561C2169080E8E0B40E1290CC
:1026820080037408F0300D077E1C7F4E122561C254
:10269200169080E8E0B4060F20160C300D077E1C61
:1026A2007F59122561D216C200050B20160302279C
:1026B20037201207122C0B8F268003E4F526E5261D
:1026C2006052300D127E1C7F6F1225617E687FA7DB
:1026D200E4FBAD2612285CE5E92410F5EB30D708BF
:1026E200E5F92428F5FB8006E5F92427F5FB906837
:1026F200A763A2019067A163A201AF26121D5485B0
:10270200260FE4F512D290C291D212C296C299203B
:1027120099FDD299122CE78F14E5146018122950F2
:10272200300D127E1C7F741225617E687FA7E4FB48
:10273200AD1412285C301008209705C210123953CC
:1027420030130A30DA07C2DAC21312395330120CCC
:0F275200E50BD394144008C212D21822E4F50B01
:012761002255
:0A395D00201604122CE7227F00223E
:103942003016037F0022301805C2187F01227F0043
:013952002252
:103110000208A4E493A3F8E493A34003F68001F229
:1031200008DFF48029E493A3F85407240CC8C333C0
:10313000C4540F4420C8834004F456800146F6DF8F
:10314000E4800B01020408102040809038C3E47E24
:10315000019360BCA3FF543F30E509541FFEE49384
:10316000A360010ECF54C025E060A840B8E493A34B
:10317000FAE493A3F8E493A3C8C582C8CAC583CA76
:10318000F0A3C8C582C8CAC583CADFE9DEE780BE2E
:0138DE0000E9
:10175100BC000BBE0029EF8DF084FFADF022E4CC7C
:10176100F875F008EF2FFFEE33FEEC33FCEE9DEC45
:10177100984005FCEE9DFE0FD5F0E9E4CEFD22ED8B
:10178100F8F5F0EE8420D21CFEADF075F008EF2FD5
:10179100FFED33FD4007985006D5F0F222C398FDC6
:0517A1000FD5F0EA2263
:1017A600E88FF0A4CC8BF0A42CFCE98EF0A42CFCE2
:1017B6008AF0EDA42CFCEA8EF0A4CDA8F08BF0A460
:1017C6002DCC3825F0FDE98FF0A42CCD35F0FCEBBF
:1017D6008EF0A4FEA9F0EB8FF0A4CFC5F02ECD3984
:0F17E600FEE43CFCEAA42DCE35F0FDE43CFC22F1
:1017F50075F008758200EF2FFFEE33FECD33CDCCAB
:1018050033CCC58233C5829BED9AEC99E58298402D
:101815000CF582EE9BFEED9AFDEC99FC0FD5F0D60A
:10182500E4CEFBE4CDFAE4CCF9A88222B800C1B934
:101835000059BA002DEC8BF084CFCECDFCE5F0CB72
:10184500F97818EF2FFFEE33FEED33FDEC33FCEBAB
:1018550033FB10D703994004EB99FB0FD8E5E4F966
:10186500FA227818EF2FFFEE33FEED33FDEC33FC53
:10187500C933C910D7059BE99A4007EC9BFCE99A47
:10188500F90FD8E0E4C9FAE4CCFB2275F010EF2F8C
:10189500FFEE33FEED33FDCC33CCC833C810D7078C
:1018A5009BEC9AE899400AED9BFDEC9AFCE899F8C7
:0E18B5000FD5F0DAE4CDFBE4CCFAE4C8F9225A
:0E18C300C3E49FFFE49EFEE49DFDE49CFC2236
:1018D100EB9FF5F0EA9E42F0E99D42F0E89C45F06D
:0118E10022E4
:0C18E200ECF0A3EDF0A3EEF0A3EFF02279
:1018EE00A8828583F0D083D08212190512190512B1
:1018FE001905121905E473E493A3C583C5F0C583D6
:10190E00C8C582C8F0A3C583C5F0C583C8C582C843
:01191E0022A6
:1013F500E53A242EF8E6053A22782B302002782E9D
:10140500E475F00112197702191F2019EB7F2ED20E
:10141500198018EF540F2490D43440D4FF301D0B9D
:10142500EF24BFB41A0050032461FFE53B600215A9
:101435003B053EE53E7002053D30200D782BE475F9
:10144500F001121977EF0219650237837403D22070
:101455008003E4C220F53A8B2B8A2C892DE4F53BD9
:10146500F53DF53EE53B60077F2012143080F575AC
:101475003CFFC21AC219C21BC21CC21EC21FC22116
:101485001213FEFF700D3020057F00121441AF3E90
:10149500AE3D22B4255FC2D5C21D1213FEFF24D076
:1014A500B40A00501A75F00A783B30D50508B6FF26
:1014B5000106C6A426F620D5047002D21C80D924C4
:1014C500CFB41A00EF5004C2E5D21D021641D21A5C
:1014D50080C6D21980C0D21B80BCD2D580BAD21E9C
:1014E50080B47F20121430201B077401B53B0040E7
:1014F500F11213F5FF121430021469D221D21F80A4
:10150500951213F5FB1213F5FA1213F5F94A4B7000
:101515000679127A177BFF201B2EE53B602A7E0099
:101525008E8275830012193860060EEE653C70F0E8
:10153500C2D5EBC0E0EAC0E0E9C0E0EE121688D003
:10154500E0F9D0E0FAD0E0FB12191FFF60AAEBC06A
:10155500E0EAC0E0E9C0E0121430D0E02401F9D09F
:10156500E03400FAD0E0FBE53C0460DCD53CD980F2
:10157500877BFF7A167984D21B809C79108002794B
:1015850008C21FC2218008D2D5790A8004790AC20F
:10159500D5E53C047002F53CE4FAFDFEFF1213F5B7
:1015A500FC7B08201A131213F5FD7B1030190A1263
:1015B50013F5FE1213F5FF7B20EC3382D592D5503F
:1015C50013C3E43019069FFFE49EFEE4201A039D31
:1015D500FDE49CFCE4CBF8C21AEC700CCFCECDCC6C
:1015E500E824F8F870F38017C3EF33FFEE33FEED10
:1015F50033FDEC33FCEB33FB994002FB0FD8E9EBF1
:10160500301A05F8D0E0C448B21AC0E00AEC4D4ED5
:101615004F78207B0070C2EAB53C0040BCC0E012A8
:10162500168AD0F0D0E0201A04C4C0E0C4B21AC0B3
:10163500F0121419D0F0D5F0EB0214691219D61571
:10164500065315805814D74C14D34215844F158C66
:0F16550044158C4914EC431592551576461576BD
:101664004515764717325014DB2D14DF2E15022B47
:1016740014E323150020171B2A149B48000014FAB6
:101684003F3F3F00790AA2D5201C14301E09B9102F
:10169400020404B9080104A2D5201F025001042049
:1016A4001B68921BB53B005034C0E07F20301C19EE
:1016B4007F30A21B721F721E500F1216E1C21BC292
:1016C4001FC21EC2217F30800F301E03E9C0E0120A
:1016D4001430301E03D0E0F9D0E0B53BCC301E17F7
:1016E4007F30B9100C1214307F58301D077F78807A
:1016F40003B90803121430301B057F2D0214307F08
:10170400202021F87F2B201FF322921B80CF286EEC
:10171400756C6C2900D21A1213F5301AF8C21A78B3
:101724003B30D50108F602149B2D5043495812133F
:10173400F52403B405004001E490172D93121421FD
:0D174400743A121421D21C753B040215806A
:101E62008B2B8A2C892DE4F537F536F535F534F5CB
:101E720032F533E52F4530452E6012EBC0E0EAC063
:101E8200E0E9C0E0AB2EAA2FA930121987AB2B05CF
:101E92002DE52DAA2C7002052C14F912191FF53804
:101EA200C394094007E538D3940D40E1E538642036
:101EB20060DBE538B42D054333038016E538B42BD7
:101EC20005433301800C74FF252DF52D74FF352C4D
:101ED200F52CE53160046410703FAB2BAA2CA92DC0
:101EE20012191F64306009E531702E75310A80299C
:101EF200900001121938FF64786004EFB45813435C
:101F020033017531107402252DF52DE4352CF52C95
:101F12008007E5317003753108AB2B052DE52DAA3D
:101F22002C7002052C14F912191FF538C394614064
:101F32000AE538D3947A50035338DF74D02538F544
:101F420038C3940A400CE5389411406D74F9253871
:101F5200F538E538D39531506043330185373C85F8
:101F6200363B85353A853439AF317E00E4FCFDAB32
:101F720037AA36A935A8341217A6C8ECC8C9EDC9C4
:101F8200CAEECACBEFCBE4FCFDFEEB2538F537EE0B
:101F92003AF536ED39F535EC38F534AF37AE36ADC6
:101FA20035FCAB3CAA3BA93AA839D31218D150034D
:101FB200021F1B433304021F1BE53320E003E480AE
:101FC2002DE52F4530452E601EAB2BE52D24FFF964
:101FD200E52C34FFFAEBC0E0EAC0E0E9C0E0AB2E4A
:101FE200AA2FA930121987E53330E20774FFFFFEEA
:101FF200FDFC22E533AF37AE36AD35AC3430E1030C
:042002000218C322DB
:10191F00BB010689828A83E0225002E722BBFE02C6
:09192F00E32289828A83E49322F9
:10193800BB010CE58229F582E5833AF583E0225064
:1019480006E92582F8E622BBFE06E92582F8E222AE
:0D195800E58229F582E5833AF583E49322C8
:10196500BB010689828A83F0225002F722BBFE0161
:02197500F3225B
:10197700FAE6FB0808E6F925F0F618E6CA3AF62271
:10198700BB011A89828A83D0F0D0E0F8D0E0F9D081
:10199700E0FAD0E0FBE8C0E0C0F0021A055016E913
:1019A700F8D083D082D0E0F9D0E0FAD0E0FBC08253
:1019B700C0830219FCBBFE16E9F8D083D082D0E0C1
:0F19C700F9D0E0FAD0E0FBC082C083021A0E22F2
:1019D600D083D082F8E4937012740193700DA3A3A0
:1019E60093F8740193F5828883E4737402936860B4
:0619F600EFA3A3A380DFB4
:0919FC00EBF608EAF608E9F62210
:091A0500EBF0A3EAF0A3E9F022E2
:091A0E00EBF208EAF208E9F22209
:00000001FF
